:020000020000FC
:0200000017C027
:02000A005BC0D9
:100026004079243019120278001051E00FEF07BB17
:100036008E9A8D9A8A9A889889988B988C9800E8D7
:1000460009BF08BF05E00EBD0DEF0DBD00270CBDB5
:10005600789460FD1DC09598969AE6E2F0E0152F1B
:100066002AE064D0E00F08F4F01FC89508BA1BD048
:100076009698959AE6E2F0E0102F2AE062D0152FC6
:10008600101BE10F08F4F11FC89508BA0CD0E1CF98
:100096009698959A0FE308BB06D09598969A0FE323
:1000A60008BB01D0D6CF0F931F930FEF1AE50A9521
:1000B600F1F71A95E1F71F910F910895F8940F93B0
:1000C60084990FC06D7F9298809922C0819924C02F
:1000D600839926C00DEF0DBD00270CBD0F917894B6
:1000E600189561FDF7CF62600F931F932F93929A35
:1000F60060FDF0CF052F2FEF14E62A95F1F71A953C
:10010600E1F70A95C1F792982F911F910F91E2CFCF
:10011600523309F05395DECF513009F05A95DACFB4
:1001260060FF02C06E7FD6CF6160D4CF1F932F933E
:100136000027121B10F00395FCCF88942F911F9176
:1001460008951F932F930027222319F0010F2A9554
:08015600FBCF2F911F910895CA
:00000001FF
